:100000000C942A001895000018950000189500001F
:10001000189500001895000018950000189500002C
:10002000189500001895000018950000189500001C
:10003000189500001895000018950000189500000C
:1000400018950000189500001895000018950000FC
:10005000189500008FE58DBFC8E2E0EF4E2E88E0D6
:100060008EBFD8E0F7E05F2EEEEFF7E0A0E6B0E05D
:1000700088278D933197E9F766248CEF84BB0E9423
:10008000EB148E9A8D9A8C9A8F9AA09AA1988B983D
:100090008A9A80E08ABBA2E3B1E0E0E4F7E30E9441
:1000A0003416A99A939A959894989698979AA89A9C
:1000B0008FEF80936600A1E7B0E0ECEEF6E30E94DC
:1000C0004318A5E7B0E0E0EFF6E30E944318A9E784
:1000D000B0E0E4EFF6E30E944318ADE7B0E0E8EFEC
:1000E000F6E30E944318A1E8B0E0ECEFF6E30E94CB
:1000F0004318EAE0F4E20E941D1381E080931001AE
:1001000000911001013318F011F00C94A1000E942D
:100110002013A0E1B1E0AD90BB24A9EEB1E0AA0CA0
:10012000BB1CAA0CBB1CAA0DBB1D0E9443180E943D
:100130001D13A0E1B1E08C918F5F8C9310F40C94AF
:10014000800081E08093DC010091DC010A3018F02E
:1001500011F00C94B5000E94370BACEDB1E08C911E
:100160008F5F8C9310F40C94A4005A924A9284E608
:1001700090E0A42DB52D8D939C9382E00E942713CF
:100180005A924A9281E0A42DB52D8C9381E00E9471
:1001900027130E94C111249683E00E9423130E941A
:1001A000E5085A924A9284E690E0A42DB52D8D93ED
:1001B0009C9382E00E9427135A924A9281E0A42DD8
:1001C000B52D8C9381E00E9427130E94C1112496C3
:1001D00083E00E9423138FEF8BBB8AEF90E00E9495
:1001E000E11381E08093D8010091D801033718F022
:1001F00011F00C940D0188E0A8EDB1E0AD90BB24A6
:10020000A0E6B1E0AA0DBB1D8C93A8EDB1E08C91E6
:100210008F5F8C9310F40C94F400A5E8B0E0E0E05C
:10022000F7E30E9443188AE08093B3008091DB01DA
:100230008F7D8093DB01E8E2F5E2A3EBB0E08C91E7
:100240009927A9E8B0E00E944E1883E08093B2009D
:10025000EEECF4E2A2EBB0E08C919927ADE8B0E0CF
:100260000E944E18E6EFF4E283E090E00E945518F9
:10027000ADEAB0E00E9434160E94EA050E9493069F
:10028000A9E8B0E00D911D912D913C9142E050E024
:1002900060E070E00E948413A1EAB0E04D935D93AA
:1002A0006D937D93A5E8B0E00D911D912D913C914A
:1002B000A1EAB0E04D915D916D917C910E94091988
:1002C000A1E9B0E00D931D932D933D93E4E0F7E396
:1002D0000E941918E9E8F0E00E94B3160E94D716B0
:1002E0000E942817FF27EDE0A9E9B0E00E948219DB
:1002F000ABEDB1E08C9185FB16F40C948D01A1E976
:10030000B0E00D911D912D913C91A5EBB0E00D93C6
:100310001D932D933C930C949901A5E8B0E00D91A9
:100320001D912D913C91A5EBB0E00D931D932D9364
:100330003C93E5EBF0E00E94B3160E94D716ADE9BE
:10034000B0E00E94081783E790E0A1EBB2E08D9344
:100350009C9381E08093DC01A1EBB2E04D915C9134
:10036000ACEDB1E00D9111270417150718F011F04D
:100370000C941B050E949B11009166000F3F11F425
:100380000C94E3015A924A9284E690E0A42DB52D94
:100390008D939C9382E00E9427135A924A9281E0A7
:1003A000A42DB52D8C9381E00E9427130E94C111CA
:1003B000249683E00E9423130E94740E8FEF809393
:1003C00066000C943C01E5EBF0E0FA93EA930E949E
:1003D0009B092296ECE6F0E0FA93EA930E94580912
:1003E00022960E947E0B0091DC010A3311F00C94DE
:1003F0005D030E94C80BADE1B1E0E0E7F7E30E94C6
:1004000034165A924A9289E1A42DB52D8C9381E03D
:100410000E9427135A924A9280E0A42DB52D8C9306
:1004200081E00E942713EDE1F1E0FA93EA930E9444
:100430001F05269682E00E942313E2EFF0E00E945F
:10044000B316E8E0F7E30E9419180E94221818F08A
:1004500011F00C942D020C943502A2E1B1E0E4E815
:10046000F7E30E9434160C944B02A8EDB7E0AF936B
:10047000BF93E2EFF0E00E94B3160E94F61311E082
:1004800002E0BF91AF910E94BC18E8EDF7E0A2E155
:10049000B1E00E947D195A924A9289E1A42DB52DAE
:1004A0008C9381E00E9427135A924A9280E0A42DF7
:1004B000B52D8C9381E00E942713E2E1F1E0FA93DD
:1004C000EA930E941F05269682E00E942313EAEC1D
:1004D000F0E00E94B316ECE0F7E30E9419180E94C6
:1004E000221810F00C94B502A8EDB7E0AF93BF93BB
:1004F000EAECF0E00E94B3160E94F61311E001E06E
:10050000BF91AF910E94BC18E8EDF7E0A2E1B1E025
:100510000E947D19EAECF0E00E94B316E0E1F7E3F7
:100520000E9419180E94221810F00C94B3028CE05B
:100530000E94F013E2E1F1E0A881B9810E947D19E7
:10054000A2E1B1E0EAE8F7E30E943416E881F9811C
:10055000A2E1B1E00E9474130E947D198CE0481A58
:100560008827580A22960C94BB02A2E1B1E0ECE87D
:10057000F7E30E9434165A924A9282E3A42DB52DD5
:100580008C9381E00E9427135A924A9280E0A42D16
:10059000B52D8C9381E00E942713E2E1F1E0FA93FC
:1005A000EA930E941F05269682E00E942313A8ED7D
:1005B000B7E0AF93BF93EEEEF0E00E94B3160E9457
:1005C000F61311E001E0BF91AF910E94BC18E8ED75
:1005D000F7E0A2E1B1E00E947D19EEEEF0E00E94AA
:1005E000B316E4E1F7E30E9419180E94221810F0F4
:1005F0000C9416038CE00E94F013E2E1F1E0A88174
:10060000B9810E947D19A2E1B1E0EAE8F7E30E9416
:100610003416E881F981A2E1B1E00E9474130E94CE
:100620007D198CE0481A8827580A2296EEEEF0E0F1
:100630000E94B316E8E1F7E30E9419180E942218FD
:1006400010F00C943F038CE00E94F013E2E1F1E023
:10065000A881B9810E947D19A2E1B1E0EAE8F7E33F
:100660000E943416E881F981A2E1B1E00E9474137E
:100670000E947D198CE0481A8827580A22965A92BF
:100680004A9280E5A42DB52D8C9381E00E9427131A
:100690005A924A9280E0A42DB52D8C9381E00E945D
:1006A0002713E2E1F1E0FA93EA930E941F052696F0
:1006B00082E00E9423130C945F030E94CF0D0091EF
:1006C000DC0141E0041BAEE0B1E00C93AEE0B1E030
:1006D0008C91855F8C9381E08093D8010091D80143
:1006E000003318F011F00C948D030091D80147E00D
:1006F000040FA0E1B1E00C93AEE0B1E04C91A0E1B9
:10070000B1E05C9190E00E94AE15A8EDB1E08C9153
:100710008F5F8C9310F40C946E0381E08093100132
:1007200000911001013318F011F00C94BB03E2EFBB
:10073000F0E00E94B316E0E1F1E0A190BB24E9EE05
:10074000F1E0AA0CBB1CAA0CBB1CEA0DFB1D0E940D
:10075000B8160E94221818F011F00C94B1030C94F2
:10076000B3030C94BB03A0E1B1E08C918F5F8C9339
:1007700010F40C949003A0E1B1E08C91895F8C930C
:1007800080911001ACEDB1E0AD90BB24A0E6B1E0EA
:10079000AA0DBB1D8C93AEE0B1E04C91ACEDB1E085
:1007A000AD90BB24A0E6B1E0AA0DBB1D5C9191E029
:1007B0000E94AE150091DC01013018F011F00C948C
:1007C000E3030C94EE04ACEDB1E00D91112741E090
:1007D00050E0041B150BA6EDB1E00D931C93A6EDA4
:1007E000B1E0AD90BC90A0E6B1E0AA0DBB1D0D91AB
:1007F0001127ACEDB1E0AD90BB24A0E6B1E0AA0DAD
:10080000BB1D4D915527041B150BA4EDB1E00D93B5
:100810001C93A4EDB1E00D911C91003050E0150740
:100820001CF011F00C9416040C941D048091DB0153
:1008300080688093DB010C9422048091DB018F7728
:100840008093DB01A4EDB1E08D919C910E94541343
:10085000A4EDB1E08D939C93A4EDB1E00D911C91BA
:10086000003050E015071CF011F00C9439040C9482
:10087000EE04A4EDB1E00D911C9142E050E00E9425
:100880003413A6EDB1E04D935C93A4EDB1E00D916E
:100890001C91A6EDB1E04D915C91041B150BA4EDEC
:1008A000B1E00D931C938091D6018093DA01ACEDF9
:1008B000B1E00D91112741E050E0041B150BA6EDAE
:1008C000B1E00D931C93A6EDB1E0AD90BC90A0E615
:1008D000B1E0AA0DBB1D8C918093D901AEE0B1E0CF
:1008E0008C9181508C930091DA01003018F011F056
:1008F0000C947C040C94AC0481E08093D80140916A
:10090000DA010091D801041718F011F00C94AC042E
:10091000ABEDB1E08C9187FB16F00C949604A9ED39
:10092000B1E08C9181508C930C949B04A9EDB1E0C3
:100930008C918F5F8C93AEE0B1E04C91A9EDB1E06A
:100940005C9191E00E94AE15A8EDB1E08C918F5FB3
:100950008C9310F40C947F04AEE0B1E08C918F5F27
:100960008C938091D4018093DA010091DA010030F8
:1009700018F011F00C94BE040C94EE0481E0809306
:10098000D8014091DA010091D801041718F011F054
:100990000C94EE04ABEDB1E08C9187FB16F00C9457
:1009A000D804A9EDB1E08C9181508C930C94DD04B6
:1009B000A9EDB1E08C918F5F8C93AEE0B1E04C91EA
:1009C000A9EDB1E05C9191E00E94AE15A8EDB1E017
:1009D0008C918F5F8C9310F40C94C104ABEDB1E05B
:1009E0008C9185FB16F40C941305E9E9F0E00E9464
:1009F000B816EDE9F0E00E94B3160E94BE17FF277B
:100A0000EDE0ADE9B0E00E948219EDE9F0E00E946E
:100A10004A1BFF27EDE00E947516A5EBB0E0EDE064
:100A2000FF270E948219ACEDB1E08C918F5F8C930F
:100A300010F40C94AC010C943C01F894FFCF81E0CD
:100A40000E94F01381E00E94F01382E00E94F013F4
:100A500081E00E94F01381E00E94F01381E00E9487
:100A6000F01381E00E94F01381E00E94F013A88946
:100A7000B9890E94B319AC85BD858C9381E0AE85A0
:100A8000BF858C93AC85BD854C91AE85BF850C919F
:100A9000041718F011F00C94E405AE85BF858C9115
:100AA000E889F98901E00A93AB85BC850E94881921
:100AB000A2E3B1E0EA85FB85222791E00E944A1675
:100AC000A885B9850C93A885B9850C91003011F0E3
:100AD0000C946E0581E0A885B9858C93A885B985AD
:100AE0008C9181508C93A885B9850C9145E0049F29
:100AF000AE81BF810C9280E080930A0100910A01CF
:100B0000043018F011F00C94DC05E4E5F5E2AE8158
:100B1000BF818C919927A885B9850E944B1880E1E7
:100B2000AA81BB818C9380E080930B0100910B0123
:100B3000043018F011F00C94CA05A885B9850C9101
:100B4000AA81BB814C910423AC81BD810C93AA89FD
:100B5000BB890C9140910B01040FA881B9810C93C2
:100B6000AC89BD894C91A881B9815C91AC81BD8172
:100B70009C910E94AE15AA81BB810C9142E00E941B
:100B8000A3190C93ABE0B1E08C918F5F8C9310F4C0
:100B90000C949605AC89BD898C918F5F8C93AE8146
:100BA000BF818C918F5F8C93AAE0B1E08C918F5FB5
:100BB0008C9310F40C947E05AE85BF858C918F5F6D
:100BC0008C9310F40C94420589E0481A8827580A3F
:100BD000609608958AE08A9387E08A938EE78A93E5
:100BE00087E08A938FEF8A930E94D5158EE78A93C8
:100BF00087E08A938EE78A9389E38A938FEF8A93BB
:100C00000E94D5158EE78A9389E38A938AE08A93B6
:100C100089E38A938FEF8A930E94D5158AE08A939D
:100C200089E38A938AE08A9387E08A938FEF8A9395
:100C30000E94D51549E058E091E00E94AE1549E0C8
:100C400056E191E00E94AE1549E050E291E00E9429
:100C5000AE1549E055E291E00E94AE1549E05AE236
:100C600091E00E94AE1549E053E391E00E94AE1579
:100C700049E058E391E00E94AE154BE05AE391E061
:100C80000E94AE1548E25AE391E00E94AE1544E49A
:100C90005AE391E00E94AE1541E65AE391E00E94CA
:100CA000AE154DE75AE391E00E94AE154FE758E0CC
:100CB00091E00E94AE154FE756E191E00E94AE151B
:100CC0004FE750E291E00E94AE154FE755E291E008
:100CD0000E94AE154FE75AE291E00E94AE154FE731
:100CE00053E391E00E94AE154FE758E391E00E9474
:100CF000AE154BE056E091E00E94AE1548E256E09A
:100D000091E00E94AE1544E456E091E00E94AE15D9
:100D100041E656E091E00E94AE154DE756E091E0C5
:100D20000E94AE150895A9E8B0E00D911D912D9196
:100D30003C9142E050E060E070E00E948413A1EA40
:100D4000B0E04D935D936D937D93A5E8B0E00D9178
:100D50001D912D913C91A1EAB0E04D915D916D9175
:100D60007C910E940919A1E9B0E00D931D932D9388
:100D70003D93A9E8B0E00D911D912D913C9144E186
:100D800050E060E070E00E948413A5E9B0E04D936C
:100D90005D936D937D93ABEDB1E08C9185FB16F483
:100DA0000C94FC06A1E9B0E00D911D912D913C91B0
:100DB0004AE050E060E070E00E948413A1E9B0E0F6
:100DC0004D935D936D937D93ADE1B1E0E1E9F0E08A
:100DD0000E942419EDE1F1E0A8EDB7E00E947D1931
:100DE000E8EDF7E0A2E1B1E01127222704E032E0CC
:100DF0000E9471180C940207A2E1B1E0E2E9F7E366
:100E00000E9434165A924A9280E0A42DB52D8C93FC
:100E100081E00E9427135A924A928BE3A42DB52DAC
:100E20008C9381E00E942713E2E1F1E0FA93EA93C8
:100E30000E941F05269682E00E942313ABEDB1E0CD
:100E40008C9185FB16F40C943B07A1E9B0E00D9161
:100E50001D912D913C91A5E9B0E04D915D916D9171
:100E60007C910E940419A1E9B0E00D931D932D938C
:100E70003D930C944D07A5E8B0E00D911D912D9187
:100E80003C914AE050E060E070E00E948413A1E9E8
:100E9000B0E04D935D936D937D93ADE1B1E0E1E9F9
:100EA000F0E00E942419EDE1F1E0A8EDB7E00E9426
:100EB0007D19E8EDF7E0A2E1B1E01127222704E077
:100EC00032E00E9471185A924A9288E3A42DB52DFF
:100ED0008C9381E00E9427135A924A928BE3A42DAF
:100EE000B52D8C9381E00E942713E2E1F1E0FA93A3
:100EF000EA930E941F05269682E00E942313ABED21
:100F0000B1E08C9185FB16F40C94B207A1E9B0E036
:100F10000D911D912D913C91A5E9B0E04D915D9110
:100F20006D917C910E940419A1E9B0E00D931D938D
:100F30002D933D93ADE1B1E0E1E9F0E00E94241989
:100F4000EDE1F1E0A8EDB7E00E947D19E8EDF7E0F2
:100F5000A2E1B1E01127222704E032E00E947118DB
:100F60000C94B807A2E1B1E0E2E9F7E30E9434167D
:100F70005A924A9286E6A42DB52D8C9381E00E9468
:100F800027135A924A928BE3A42DB52D8C9381E0BE
:100F90000E942713E2E1F1E0FA93EA930E941F0511
:100FA000269682E00E942313ADE1B1E0E8E9F7E381
:100FB0000E9434165A924A9283E0A42DB52D8C9348
:100FC00081E00E9427135A924A9283E2A42DB52D04
:100FD0008C9381E00E942713EDE1F1E0FA93EA930C
:100FE0000E941F05269682E00E942313ADE1B1E026
:100FF000EAE9F7E30E9434165A924A9283E0A42D5C
:10100000B52D8C9381E00E9427135A924A9288E270
:10101000A42DB52D8C9381E00E942713EDE1F1E022
:10102000FA93EA930E941F05269682E00E942313FA
:10103000ADE1B1E0ECE9F7E30E9434165A924A922E
:1010400083E0A42DB52D8C9381E00E9427135A9242
:101050004A9281E3A42DB52D8C9381E00E94271341
:10106000EDE1F1E0FA93EA930E941F05269682E0F3
:101070000E942313ADE1B1E0EEE9F7E30E943416DC
:101080005A924A9280E0A42DB52D8C9381E00E9463
:1010900027135A924A9286E0A42DB52D8C9381E0B5
:1010A0000E942713EDE1F1E0FA93EA930E941F05F5
:1010B000269682E00E942313ADE1B1E0E0EAF7E377
:1010C0000E9434165A924A9280E0A42DB52D8C933A
:1010D00081E00E9427135A924A9284E1A42DB52DF3
:1010E0008C9381E00E942713EDE1F1E0FA93EA93FB
:1010F0000E941F05269682E00E942313ADE1B1E015
:10110000E2EAF7E30E9434165A924A9280E0A42D54
:10111000B52D8C9381E00E9427135A924A928EE15A
:10112000A42DB52D8C9381E00E942713EDE1F1E011
:10113000FA93EA930E941F05269682E00E942313E9
:10114000ADE1B1E0E4EAF7E30E9434165A924A9224
:1011500080E0A42DB52D8C9381E00E9427135A9234
:101160004A9285E3A42DB52D8C9381E00E9427132C
:10117000EDE1F1E0FA93EA930E941F05269682E0E2
:101180000E942313EDEAF0E0ADE1B1E00E947D1989
:101190005A924A9280E0A42DB52D8C9381E00E9452
:1011A00027135A924A9280E0A42DB52D8C9381E0AA
:1011B0000E942713EDE1F1E0FA93EA930E941F05E4
:1011C000269682E00E94231308950E94511588EC10
:1011D00090E00E94E113ADE1B1E0E6EAF7E30E949E
:1011E00034165A924A928DE1A42DB52D8C9381E04C
:1011F0000E9427135A924A9284E1A42DB52D8C9314
:1012000081E00E942713EDE1F1E0FA93EA930E9456
:101210001F05269682E00E942313ADE1B1E0E6EBC4
:10122000F7E30E9434165A924A9289E1A42DB52D13
:101230008C9381E00E9427135A924A928EE1A42D4A
:10124000B52D8C9381E00E942713EDE1F1E0FA9334
:10125000EA930E941F05269682E00E942313ADE1C7
:10126000B1E0E8ECF7E30E9434165A924A928EE11C
:10127000A42DB52D8C9381E00E9427135A924A9297
:1012800082E3A42DB52D8C9381E00E942713EDE11C
:10129000F1E0FA93EA930E941F05269682E00E94ED
:1012A0002313E2E0F0E00E947B130E9451150895A1
:1012B0008C9A8D9A9598A881B98190E28D919830F9
:1012C00018F4392F992702C038E0985087959498E0
:1012D00008F4949A00000000959A00000000959888
:1012E000000000003A9591F7992341F781E080933F
:1012F00070008C9A8D9A9598A0E7B0E098E08D9157
:10130000983018F4392F992702C038E09850879503
:10131000949808F4949A00000000959A0000000048
:101320009598000000003A9591F7992341F7969A15
:10133000000096980895A881B9810D911D912D9175
:101340003C91A9EBB0E00D931D932D933C9380E16C
:1013500097E2A1ECB0E08D939C93ACE6B0E00E94E4
:101360006118A9EBB0E00D911C91A1ECB0E04D919A
:101370005C910E945A13ADEBB0E04D935C9381E019
:1013800090E0AFEBB0E08D939C93ADEBB0E04D916E
:101390005C91AFEBB0E00D911C910417150718F0AC
:1013A00011F00C94000AACE6B0E00D911D912D9166
:1013B0003C91A1E7B0E04D915D916D917C910E94CF
:1013C0000419ACE6B0E00D931D932D933D93A9EB6A
:1013D000B0E00D911D912D913C9140E157E260E00C
:1013E00070E00E940919A9EBB0E00D931D932D93B5
:1013F0003D93AFEBB0E00E942B1310F00C94C509A5
:1014000088EE93E0A1ECB0E08D939C93A9EBB0E063
:101410000D911C91A1ECB0E04D915C910E945A138A
:10142000ADEBB0E04D935C9381E090E0AFEBB0E0CA
:101430008D939C93ADEBB0E04D915C91AFEBB0E040
:101440000D911C910417150718F011F00C94550A12
:10145000ACE6B0E00D911D912D913C91A5E7B0E077
:101460004D915D916D917C910E940419ACE6B0E0C4
:101470000D931D932D933D93A9EBB0E00D911D911C
:101480002D913C9148EE53E060E070E00E94091914
:10149000A9EBB0E00D931D932D933D93AFEBB0E01E
:1014A0000E942B1310F00C941A0A84E690E0A1EC31
:1014B000B0E08D939C93A9EBB0E00D911C91A1EC51
:1014C000B0E04D915C910E945A13ADEBB0E04D93AA
:1014D0005C9381E090E0AFEBB0E08D939C93ADEB3B
:1014E000B0E04D915C91AFEBB0E00D911C91041711
:1014F000150718F011F00C94AA0AACE6B0E00D91B3
:101500001D912D913C91A9E7B0E04D915D916D91B8
:101510007C910E940419ACE6B0E00D931D932D93CD
:101520003D93A9EBB0E00D911D912D913C9144E6C6
:1015300050E060E070E00E940919A9EBB0E00D9363
:101540001D932D933D93AFEBB0E00E942B1310F051
:101550000C946F0A8AE090E0A1ECB0E08D939C932C
:10156000A9EBB0E00D911C91A1ECB0E04D915C9124
:101570000E945A13ADEBB0E04D935C9381E090E094
:10158000AFEBB0E08D939C93ADEBB0E04D915C91EF
:10159000AFEBB0E00D911C910417150718F011F096
:1015A0000C94FF0AACE6B0E00D911D912D913C9199
:1015B000ADE7B0E04D915D916D917C910E94041971
:1015C000ACE6B0E00D931D932D933D93A9EBB0E0F5
:1015D0000D911D912D913C914AE050E060E070E04A
:1015E0000E940919A9EBB0E00D931D932D933D9333
:1015F000AFEBB0E00E942B1310F00C94C40AA9EBDF
:10160000B0E08D919C91ADEBB0E08D939C9381E027
:1016100090E0AFEBB0E08D939C93ADEBB0E04D91DB
:101620005C91AFEBB0E00D911C910417150718F019
:1016300011F00C94360BACE6B0E00D911D912D919C
:101640003C91A1E8B0E04D915D916D917C910E943B
:101650000419ACE6B0E00D931D932D933D93AFEBD1
:10166000B0E00E942B1310F00C940D0B0895ACE623
:10167000B0E00E9461188C9A8D9A9598ACE6B0E023
:1016800090E28D91983018F4392F992702C038E0F4
:1016900098508795949808F4949A00000000959AC1
:1016A000000000009598000000003A9591F79923FA
:1016B00041F780E0809370008C9A8D9A9598A0E70E
:1016C000B0E098E08D91983018F4392F992702C036
:1016D00038E098508795949808F4949A0000000098
:1016E000959A000000009598000000003A9591F747
:1016F000992341F7969A000096980895A3ECB0E0DC
:101700000E945F18A5ECB0E00E945F1880E092E0B4
:10171000A7ECB0E08D939C939798A7ECB0E00D9167
:101720001C91003050E0150718F011F00C949A0B42
:101730000C94C50BA898999B0C94AC0BA3ECB0E04F
:101740000D911C91A7ECB0E04D915C91040F151F19
:10175000A3ECB0E00D931C93839B0C94BD0BA5EC04
:10176000B0E00D911C91A7ECB0E04D915C91040F9D
:10177000151FA5ECB0E00D931C93A89A91E0A7EC7F
:10178000B0E00E943A160C948D0B979AA89A08958F
:10179000ECE1F7E30E941918E5ECF0E0D190E0806D
:1017A000FF2400270E94D7160E947E17FF27EDE036
:1017B000AAECB0E00E948219E0E2F7E30E94191857
:1017C000EAECF0E00E94B3160E94AF17FF27EDE0AD
:1017D000AAECB0E00E948219E4E2F7E30E94191833
:1017E000E3ECF0E0D190E080FF2400270E94D716C0
:1017F0000E947E17FF27EDE0AEECB0E00E94821958
:10180000E8E2F7E30E941918EAECF0E00E94B31650
:101810000E942817FF27EDE0AEEFB0E00E9482198A
:10182000A2E0B1E0ECE2F7E30E944318E2E0F1E06D
:10183000AEEFB0E00E940D1BFF27EDE0A2EDB0E09F
:101840000E948219E2EDF0E00E94B816E0E3F7E3AF
:101850000E9410180E942817FF27EDE0A2EDB0E0CB
:101860000E948219E2EDF0E00E94B816E0E3F7E38F
:101870000E9410180E94BE17FF27EDE0AEEFB0E007
:101880000E948219E2EDF0E00E94B816E0E3F7E36F
:101890000E9410180E94AF17FF27EDE0A2E0B1E010
:1018A0000E948219E2E0F1E00E94B816EEEFF0E04B
:1018B0000E94B3160E942817FF27EDE0A6E0B1E0D2
:1018C0000E948219E6E0F1E00E94B919FF27EDE0DD
:1018D000A2EFB0E00E948219E4E3F7E30E94191836
:1018E000EEECF0E00E94B3160E942817FF27EDE00F
:1018F000AEEFB0E00E948219EEEFF0E00E94D8193E
:10190000FF27EDE0A6EDB0E00E948219EEEFF0E0D7
:101910000E942F1BFF27EDE0AAEDB0E00E94821984
:10192000E2EDF0E00E94B816E6EDF0E00E94B3169A
:101930000E947E17FF27EDE0AEEDB0E00E94821915
:10194000E2EDF0E00E94B816EAEDF0E00E94B31676
:101950000E947E17FF27EDE0A2EEB0E00E94821900
:10196000EEEDF0E00E94B816E0E3F7E30E941018F5
:101970000E94AF17FF27EDE0AEEFB0E00E948219A2
:10198000EEEFF0E00E94B816EEEFF0E00E94B31622
:101990000E947E17FF27EDE0A6EFB0E00E948219BB
:1019A000E2EEF0E00E94B816E2EEF0E00E94B3161C
:1019B0000E947E17FF27EDE0AAEFB0E00E94821997
:1019C000EAEFF0E00E94B816E6EFF0E00E94B316EE
:1019D0000E94BE17FF27EDE0AEEFB0E00E94821933
:1019E000E2EEF0E00E94B816E8E3F7E30E94101878
:1019F0000E947E17FF27EDE0A2E0B1E00E9482196D
:101A0000EEEFF0E00E94B816E2E0F1E00E94B316BB
:101A10000E942817FF27EDE0A6E0B1E00E9482199E
:101A2000ECE3F7E30E941918E6E0F1E00E94B31638
:101A30000E947E17FF27EDE0AEEFB0E00E94821912
:101A4000EEEFF0E00E94B919FF27EDE0A6EEB0E05E
:101A50000E948219EEEDF0E00E94B816EEEDF0E083
:101A60000E94B3160E947E17FF27EDE0AEEFB0E0B4
:101A70000E948219EEEFF0E00E94B816E0E3F7E36F
:101A80000E9410180E94AF17FF27EDE0A2E0B1E01E
:101A90000E948219EAEFF0E00E94B816E2E0F1E05D
:101AA0000E94B3160E94AF17FF27EDE0AEEFB0E043
:101AB0000E948219EAEFF0E00E94B816E6EFF0E02B
:101AC0000E94B3160E94BE17FF27EDE0A2E0B1E02E
:101AD0000E948219E2E0F1E00E94B816EEEFF0E019
:101AE0000E94B3160E942817FF27EDE0A6E0B1E0A0
:101AF0000E948219ECE3F7E30E941918E6E0F1E096
:101B00000E94B3160E947E17FF27EDE0AEEFB0E013
:101B10000E948219EEEFF0E00E94B919FF27EDE074
:101B2000AAEEB0E00E948219EAEEF0E00E94B81638
:101B3000EAEEF0E00E94B3160E947E17FF27EDE068
:101B4000AEEFB0E00E948219E6EEF0E00E94B81617
:101B5000E6EEF0E00E94B3160E947E17FF27EDE04C
:101B6000A2E0B1E00E948219E2E0F1E00E94B81622
:101B7000EEEFF0E00E94B3160E94BE17FF27EDE0E3
:101B8000A6E0B1E00E948219E6E0F1E00E94541B59
:101B9000FF27EDE0AEEEB0E00E9482190895ECE17F
:101BA000F7E30E941918E5ECF0E0D190E080FF2403
:101BB00000270E94D7160E947E17FF27EDE0AAECAF
:101BC000B0E00E948219E0E2F7E30E941918EAEC03
:101BD000F0E00E94B3160E94AF17FF27EDE0AAECD9
:101BE000B0E00E948219E4E2F7E30E941918E3ECE6
:101BF000F0E0D190E080FF2400270E94D7160E94D9
:101C00007E17FF27EDE0AEECB0E00E948219E8E21B
:101C1000F7E30E941918EAECF0E00E94B3160E9464
:101C20002817FF27EDE0AEEFB0E00E948219A2E096
:101C3000B1E0ECE2F7E30E944318E2E0F1E0AEEF3E
:101C4000B0E00E940D1BFF27EDE0A2EDB0E00E9486
:101C50008219E2EDF0E00E94B816E0E3F7E30E949B
:101C600010180E942817FF27EDE0A2EDB0E00E94B7
:101C70008219E2EDF0E00E94B816E0E3F7E30E947B
:101C800010180E94BE17FF27EDE0AEEFB0E00E94F3
:101C90008219E2EDF0E00E94B816E0E3F7E30E945B
:101CA00010180E94AF17FF27EDE0A2E0B1E00E94FC
:101CB0008219E2E0F1E00E94B816EEEFF0E00E9437
:101CC000B3160E942817FF27EDE0A6E0B1E00E94BE
:101CD0008219E6E0F1E00E94B919FF27EDE0A2EFDA
:101CE000B0E00E9482190895009166000D3F11F046
:101CF0000C94F60EA9E8B0E00D911D912D913C9148
:101D000042E050E060E070E00E948413A1EAB0E09D
:101D10004D935D936D937D93A5E8B0E00D911D917A
:101D20002D913C91A1EAB0E04D915D916D917C9136
:101D30000E940419A1EAB0E00D931D932D933D93E9
:101D4000A1EAB0E00D911D912D913C91ADE8B0E07C
:101D50004D915D916D917C910E940419A1EAB0E0D2
:101D60000D931D932D933D9340E65AEE60E070E095
:101D7000A1EAB0E00D911D912D913C910E940E19A8
:101D80001CF011F00C94C60E0C94E20E5A924A927A
:101D900082E390E0A42DB52D8D939C9382E00E9468
:101DA00027135A924A9282E0A42DB52D8C9381E09C
:101DB0000E9427130E94C111249683E00E942313DE
:101DC0000C94F60EA5E8B0E00D911D912D913C917B
:101DD000ADE8B0E04D915D916D917C910E94041948
:101DE000A5E8B0E00D931D932D933D9300916600FF
:101DF0000E3F11F00C94760FA9E8B0E00D911D9103
:101E00002D913C9142E050E060E070E00E9484132C
:101E1000A1EAB0E04D935D936D937D93A5E8B0E0AA
:101E20000D911D912D913C91A1EAB0E04D915D91F4
:101E30006D917C910E940919A1EAB0E00D931D9368
:101E40002D933D93A1EAB0E00D911D912D913C9110
:101E5000ADE8B0E04D915D916D917C910E940919C2
:101E6000A1EAB0E00D931D932D933D9348EE53E00E
:101E700060E070E0A1EAB0E00D911D912D913C91E0
:101E80000E940E190CF402C00C94620F5A924A92EE
:101E900082E390E0A42DB52D8D939C9382E00E9467
:101EA00027135A924A9282E0A42DB52D8C9381E09B
:101EB0000E9427130E94C111249683E00E942313DD
:101EC0000C94760FA5E8B0E00D911D912D913C91F9
:101ED000ADE8B0E04D915D916D917C910E94091942
:101EE000A5E8B0E00D931D932D933D9300916600FE
:101EF000073F11F00C9452108091DB018F7D80938D
:101F0000DB010091B3000A3011F00C94A30F5A9238
:101F10004A9282E390E0A42DB52D8D939C9382E0AC
:101F20000E9427135A924A9282E0A42DB52D8C93D9
:101F300081E00E9427130E94C111249683E00E9431
:101F400023130C9452100091B30041E0040FA4EB52
:101F5000B0E00C93E8E2F5E2A4EBB0E08C919927B5
:101F6000A9EAB0E00E944E18A9EAB0E00D911D91D7
:101F70002D913C9142E050E060E070E00E948413BB
:101F8000A1EAB0E04D935D936D937D93A5E8B0E039
:101F90000D911D912D913C91A1EAB0E04D915D9183
:101FA0006D917C910E940919A1EAB0E00D931D93F7
:101FB0002D933D93A9EAB0E00D911D912D913C9197
:101FC00042E050E060E070E00E948413A5EAB0E0D7
:101FD0004D935D936D937D93A5E8B0E00D911D91B8
:101FE0002D913C91A5EAB0E04D915D916D917C9170
:101FF0000E940419A5EAB0E00D931D932D933D9323
:1020000048EE53E060E070E0A1EAB0E00D911D9170
:102010002D913C910E940E1980E00CF481E08F9389
:1020200040E65AEE60E070E0A5EAB0E00D911D9147
:102030002D913C910E940E1980E014F009F081E08E
:102040009F91892B882311F40C9442105A924A9242
:1020500082E390E0A42DB52D8D939C9382E00E94A5
:1020600027135A924A9282E0A42DB52D8C9381E0D9
:102070000E9427130E94C111249683E00E9423131B
:102080000C9452108091B4008093B300A9EAB0E0A0
:102090000D911D912D913C91A9E8B0E00D931D93F8
:1020A0002D933C93009166000B3F11F00C9414119A
:1020B0000091B300003011F00C9465108091DB01A9
:1020C00080628093DB010C9414110091B30041E015
:1020D000041BA4EBB0E00C93E8E2F5E2A4EBB0E063
:1020E0008C919927A9EAB0E00E944E18A9EAB0E0C5
:1020F0000D911D912D913C9142E050E060E070E027
:102100000E948413A1EAB0E04D935D936D937D939B
:10211000A5E8B0E00D911D912D913C91A1EAB0E0B0
:102120004D915D916D917C910E940919A1EAB0E0F9
:102130000D931D932D933D93A9EAB0E00D911D9150
:102140002D913C9142E050E060E070E00E948413E9
:10215000A5EAB0E04D935D936D937D93A5E8B0E063
:102160000D911D912D913C91A5EAB0E04D915D91AD
:102170006D917C910E940419A5EAB0E00D931D9326
:102180002D933D9348EE53E060E070E0A1EAB0E0AB
:102190000D911D912D913C910E940E1980E00CF43F
:1021A00081E08F9340E65AEE60E070E0A5EAB0E08F
:1021B0000D911D912D913C910E940E1980E014F01B
:1021C00009F081E09F91892B882311F40C9404116C
:1021D0005A924A9282E390E0A42DB52D8D939C9360
:1021E00082E00E9427135A924A9282E0A42DB52DD4
:1021F0008C9381E00E9427130E94C111249683E0F2
:102200000E9423130C9414118091B4008093B300A6
:10221000A9EAB0E00D911D912D913C91A9E8B0E0A3
:102220000D931D932D933C93009166000F3D11F08B
:102230000C9457110091B200093011F00C943C112C
:102240005A924A9282E390E0A42DB52D8D939C93EF
:1022500082E00E9427135A924A9282E0A42DB52D63
:102260008C9381E00E9427130E94C111249683E081
:102270000E9423130C945711A2EBB0E08C918F5F56
:102280008C93EEECF4E2A2EBB0E08C919927ADE8F0
:10229000B0E00E944E18E6EFF4E2A2EBB0E08C91C1
:1022A00099270E945518ADEAB0E00E9434160091BB
:1022B00066000F3E11F00C949A110091B2000030AC
:1022C00011F00C947F115A924A9282E390E0A42D6F
:1022D000B52D8D939C9382E00E9427135A924A92C7
:1022E00082E0A42DB52D8C9381E00E9427130E94DB
:1022F000C111249683E00E9423130C949A11A2EB3F
:10230000B0E08C9181508C93EEECF4E2A2EBB0E063
:102310008C919927ADE8B0E00E944E18E6EFF4E208
:10232000A2EBB0E08C9199270E945518ADEAB0E07D
:102330000E9434160895A5E6B0E089B38C9300910D
:1023400065000F3F11F40C94C011809165008093DB
:10235000660089E190E00E94E11380E080936500CF
:10236000009165000F3F11F40C94BC11A5E6B0E09C
:1023700089B38C930C94B01189E190E00E94E11331
:10238000089581E090E0A7E6B0E08D939C93AA8148
:10239000BB814D915C91A7E6B0E00D911C910417B3
:1023A000150718F011F00C940212BB27A2E38C91D0
:1023B00082FB882780F9809580FBBB27A2E38C9164
:1023C00082F98C93A881B9818C9199270E94E1139D
:1023D000BB27A2E38C9182FB882780F9809580FB44
:1023E000BB27A2E38C9182F98C93A881B9818C914F
:1023F00099270E94E113A7E6B0E00E942B1310F08A
:102400000C94C7110895F894FFCF588A6042158C38
:102410000E427502B841D8F07641C4423041C18BBA
:1024200007417F6ADF40D786C140C251AC400517E3
:102430009B4086C98B40D39F7B404278624083A3F8
:102440004C40F4893A40C53D2C40E6742140B79C8D
:10245000194098FA1340E6CB0F404E620C40A83565
:10246000094029ED0540B35E0240A110FD3F790609
:10247000F53F3EEDEC3F3815E53F5EBADD3F38F8FD
:10248000D63F8AC8D03F9E07CB3F5183C53F1B0D27
:10249000C03FC68ABA3F8104B53F8BA6AF3FAEB6F8
:1024A000AA3F077CA63FB116A33F8F53A03F5A8196
:1024B0009D3F9560993F4547923FCDCC8C3F6666E6
:1024C000863F0AD7833FAE47813F0000803F0A0026
:1024D0000000140000003200000064000000C8008A
:1024E0000000F4010000E8030000D007000088139A
:1024F0000000102700002031304B002032304B000C
:102500002035304B003130304B003230304B00350D
:1025100030304B002020314D002020324D00202053
:10252000354D002031304D00140000003200000015
:1025300064000000C8000000F4010000E80300008F
:10254000D00700008813000010270000204E000074
:1025500050C300000008101508000304081000080C
:102560001F1F0800021F1F020000000000000001E2
:102570000000000004040400000B150900001D15F4
:10258000120000101718000E11110E00091F010093
:10259000000B151509000A11150E00060A1F02008E
:1025A0001D15151200020D15020010131418000A53
:1025B00015150A000815160C000F14140F001F152E
:1025C000150A000E111111001F11110E001F151117
:1025D00011001F141010000E111517001F04041F06
:1025E00000111F1100001211111E001F040A11001A
:1025F0001F010101001F18181F001F18061F000EE1
:1026000011110E001F141408000E11130F001F14D7
:102610001609000915151200101F1000001E0101F7
:102620001E001C02011E001F03031F00110A0619D1
:1026300000110A041800131515198E2E9F2E0895E7
:10264000E82DF92D0895481A8827580A0895480E4C
:102650008827581E0895ED91FC913196FC93EE93D6
:10266000089500FC10D0089503D024D001F8F9CFCC
:102670000024E89457FF02C009D0689400F80BD0FA
:1026800010F80124089502D009D00895509540957E
:102690004F5F5F4F0895E89417FF089500951095D8
:1026A0000F5F1F4F6894089599231AF480959095B1
:1026B00001960895352F242FE894452B11F4689442
:1026C0000895512F402F0027112780E1440F551FF7
:1026D000001F111F021B130B416018F4020F131F80
:1026E0004E7F8A9599F708958F938D918823E9F706
:1026F00011978F91089588EE93E063D03197D9F7C1
:10270000089500FC05D0089530D005D001F8F9CF28
:1027100037D03FD00895842F952FA62FB72FE89458
:10272000452B462B472B11F468940895402F512FC9
:10273000622F732F0027112722273327F0E2440F3F
:10274000551F661F771F001F111F221F331F081BF5
:10275000190B2A0B3B0B416028F4080F191F2A1F85
:102760003B1F4E7FFA9559F708950024E89477FFB0
:1027700002C006D0689400F809D010F8012408952A
:1027800012D04F5F5F4F6F4F7F4F0895E89437FF30
:10279000089500951095209530950F5F1F4F2F4F8E
:1027A0003F4F6894089540955095609570950895B1
:1027B0003197F1F70895689462F80895E89462F803
:1027C0000895EF93FF93EE27E82BE92B31F0E0ED2E
:1027D000F7E03197F1F70197D1F7FF91EF91089565
:1027E0005A924A92480E8827581E08958DE207FD96
:1027F0008D938F2D881F802F881F8F57082F6894E7
:10280000F7F8802F87FF15C080958395082F80E308
:102810008D938EE28D93802F815228F080E38D93EB
:1028200099279C93089544270A95802F09F196D003
:102830001FC0805230F09EE49D9381E48D939D9360
:10284000EFCF4427DF92EF92FF920F938FE1801B2F
:1028500011F0082F83D089D09EE29D930F91FF90B5
:10286000EF90DF9044270395003209F4D7CF2BD0A7
:102870003F93ECEFF8E238E12F2D1E2D0D2DFF24B4
:10288000EE24DD244427000F111F221FA8F42F92ED
:102890003F920E940C18102C0E940C18202C0E94B1
:1028A0000C18302C0E940C183197410DD21CE31CDF
:1028B000F01C3F902F9001C0339631963A9519F74E
:1028C0003F9107D0AFCFDD0CEE1CFF1C0A95D9F766
:1028D0000895002719E058D08F93802B11F00395AD
:1028E00001C08F911A95B9F7802F882309F496CFEC
:1028F0008F91805D8D930A95D9F792CF0065CD1D9C
:1029000080B2E60E40597307A0ACB90350D6DC0183
:10291000286BEE0094357700CA9A3B0065CD1D0008
:10292000B2E60E0059730700ACB90300D6DC010013
:102930006BEE0000357700009A3B0000CD1D0000D3
:10294000E60E000073070000B9030000DC01000080
:10295000EE000000770000003B000000F694E794D2
:10296000D79447950A95D1F7089500270DD08F93F6
:1029700003958F2D8E298D29842BC1F78F91805D32
:102980008D930A95D9F74CCF1F930F93002710E230
:10299000440FDD1CEE1CFF1C001F802F9AE0890BEA
:1029A00010F0082F43951A9599F7802F0F911F91DA
:1029B00008952093B7023093B8024093B902509320
:1029C000BA0208952091B7023091B8024091B9023D
:1029D0005091BA020895442719D0AD98AC9AAA989C
:1029E00084E699270E94E1139FEF97BBAD9A30D000
:1029F00014FCFDCF02D04FEF09D08FE310D080EC54
:102A00000ED080E40CD088EB0AD00895403420F03A
:102A1000AF9AAE9840540895AE9AAF980895AB9887
:102A200001C0AB9AEF93FF93E6E0F0E00E94D81369
:102A3000FF91EF9188BBAC98AA9A000000000000BB
:102A4000000000000000000000000000AA980895A7
:102A5000AB9804D017FCFCCF0895AB9A992797BB8D
:102A60009FEF98BBEF93FF93E6E0F0E00E94D8134E
:102A7000FF91EF91AC9AAA9A0000000000000000BC
:102A80000000000000000000000000000000000046
:102A90000000000000000000000016B2AA9897BBDA
:102AA00008954427B3DF02D04FEFB0DF00E080E4A9
:102AB000B6DF88EB800FB3DF10E48827B2DF1A950A
:102AC000E1F70395083099F70895EF93FF9350913C
:102AD00062005F9370906300E0916000F09161008C
:102AE0000E940C18202D0E940C18302D0E940C18EA
:102AF000002D31968052482F0E949719E40FF51F40
:102B000070926300732F40916300509162001DD05A
:102B10000E940C18802D50916400552309F0809577
:102B200080DF509163005395509363007A9559F775
:102B3000509162005395509362002A9509F75F9176
:102B400050936200FF91EF9108954A955A955EDF88
:102B500088EB850F64DF80E4840F61CF0F921F92B2
:102B60002F923F920F939F934F93052F48E00E941F
:102B7000A319082E4F91502F242E352EE8DF6DDF3C
:102B80006CDF422D532DE3DF802D0E9467180F91DB
:102B9000002311F0182A01C01922812D42DF0F9164
:102BA0003F902F901F900F900895AA24BB24FF24DC
:102BB000EC81EA80EE1AFF08FB81298033242F1A6A
:102BC000330881E0EA14FA043CF42FEF3FEFE0947D
:102BD000F094E80EFA1C02C021E033272A143A04CC
:102BE0003CF46FEF7FEF20943094280E3A1C02C023
:102BF00061E0772735D02E143F0414F009F017C098
:102C0000CE2CDF2CCC0CDD1C022C132C000C111C48
:102C10009A81E91761F0E20FA00CB11CAE14BF0459
:102C200024F019F0F60FAC18BD081AD0F1CFC22C61
:102C3000D32CCC0CDD1C0E2C1F2C000C111C9981EC
:102C4000F91711F425960895F60FA00CB11CA214E3
:102C5000B30424F019F0E20FAC18BD0801D0EFCF97
:102C60004E2F5F2F98817ACF0E940C180D92002072
:102C7000D9F70895903041F00D911C911695079564
:102C80009A95E1F71C930E93089599910027A90F47
:102C9000B01F1197492F4A955E2F6F2FE894112787
:102CA0004395203019F0C895802D01C0808188237C
:102CB000B9F07C917723A1F0781739F40EF0042F46
:102CC0001395689411963196EBCF112321F0411B97
:102CD000A11B1127B10BE894E52FF62F1196E0CF39
:102CE000882311F00027089508953DD099271127D2
:102CF0008F2D880F80E8F82A802F881F08F41FEF97
:102D000041F08F57082F07FD04C0003240F08FEFCD
:102D100001C08827982FD82EE82EF82E09C08FE101
:102D2000801B082FF694E794D79497950A95D1F7CE
:102D3000112351F09095D094E094F09481E0980F95
:102D40008827D81EE81EF81E0F2DFE2CED2CD92E3C
:102D50000895D094E094F09491E0D90E9927E91E5B
:102D6000F91E10950895D190E190F1900191089588
:102D700021913191419151910895102F90E8FF0CCC
:102D8000001F0927990FF7941078652F90E8440FDA
:102D9000551F5927990F4795607800380895FF0C03
:102DA00090E89027110F9795F794092F0895102F09
:102DB000BD2CDE2CEF2CF02E11234AF4B094D094CD
:102DC000E094F0949FEFB91AD90AE90AF90A0EE1E2
:102DD000FF2039F4FE2CED2CDB2CBB240850C2F76D
:102DE0006BC032F00A95BB0CDD1CEE1CFF1CF9CF4A
:102DF00001D0D5CFB7FE089590E8B91611F4D0FEF2
:102E000008959FEFD91AE90AF90A09F4039508957C
:102E1000DD92ED92FD920C930895502F2D2D3E2DB5
:102E20004F2D612F08952DEC3CEC4CEC5DE36627B3
:102E30000FC099DFF2DFDD24EE2490E8F92E0FE3D6
:102E400007C096DF05C02227332740E251E46627FA
:102E5000552351F1002381F190DF71F116270058BD
:102E600050580894050B18F407FD03C025C007FD52
:102E700023C0469537952795F694E794D79422D0AA
:102E8000FF202AF0DD0CEE1CFF1C015073F09D2D7D
:102E9000969548F0DD203AF4EE202AF491E0D90E20
:102EA0009927E91EF91E7BCF07C09FE7092FF92A52
:102EB0009FEFD92EE92E0895DD24EE24FF2400276C
:102EC000112708959F929924AA24BB2488E1D21641
:102ED000E306F40628F0D21AE30AF40A089401C0C3
:102EE0008894991CAA1CBB1CDD0CEE1CFF1C8A9547
:102EF00071F7D92CEA2CFB2C9F9008953EDFE1F26C
:102F00005038D1F21627005850580894051F12F473
:102F100018F4CBCF08F0D0CF0AD0FF202AF0BB0C9A
:102F2000DD1CEE1CFF1C3BCF0F5FFBF138CF9F92E7
:102F30009924AA24BB24992788E1990CAA1CBB1CBC
:102F4000DD1CEE1CFF1C30F4920EA31EB41ED91E15
:102F5000E91EF91E8A9589F79F90089509DF0DDF14
:102F6000503829F090E869270CC00AF045D017CFF7
:102F70005FE322273327442701C0FADEFEDE503804
:102F8000B1F3003899F3902F951B8BF312F434D0E2
:102F9000FACF983118F0222733274427983028F0A9
:102FA000232F342F44279850F9CF992329F04695A1
:102FB000379527959A95D9F7912F962742F014D0F7
:102FC000B0F6F794E794D7940F5F8BF66ECF10D0DE
:102FD00051F008F4BEDEFF2052F2DD0CEE1CFF1CA7
:102FE0000150CBF762CF68CFD20EE31EF41E0895D6
:102FF000D21AE30AF40A0895DF92EF92FF920F9338
:103000001F93D22EE32EF42E052F162F6F915F9172
:103010004F913F912F910895C895319600200895C2
:10302000FBDFD02CF9DFE02CF7DFF02CF5DF002DF3
:103030000895F2DF202DF0DF302DEEDF402DECDFA4
:10304000502D089507FB00680EF40F7757FB50686A
:103050000EF45F7707FD02C057FF05C0D216E306E6
:10306000F406050708952D153E054F0550070895F0
:1030700000240D280E280F28002A0020089591E032
:1030800005C092E003C094E001C098E0C5DF0D9256
:103090009A95E1F70895E80FF91FF1CF880F991F6E
:1030A000880F991FE80FF91FEECF882311F4992399
:1030B00029F00E940C18E9F70197D9F7089582E0EA
:1030C00001C084E099279D938A95E9F7089591E0DE
:1030D000882321F08894991F8A95E9F7892F909584
:1030E00008952E2E3F2E992781918D3209F09395C8
:1030F0008823D1F79A95E22DF32D112361F009175A
:1031000018F011F0101B01C0191B28F021F080E20B
:103110008D931A95E9F780818D3219F48D9331964C
:1031200004C0222311F08BE28D93091738F031F09F
:10313000091B21F080E38D930A95E9F781918D9326
:103140008823E1F7332351F0EA2FFB2F3196339593
:103150008E9182933A95E1F78EE28C9308959927A8
:103160008D9193958823E1F7939511968C93119700
:103170008E919A95D1F70895EA2FFB2F00244C9158
:103180008D9103948E32E1F711248D91139488234D
:10319000E1F71A94101640F41197202F2119239566
:1031A00080E38D932A95E9F7113039F59927AE2FF1
:1031B000BF2FA00DB91FA00FB91F8C919C93853311
:1031C00008F421C031E08E918E32E9F38D3241F066
:1031D000830F8A3319F480E331E001C033278C93E5
:1031E000AE1789F7332341F0AE2FBF2FB8DF81E34D
:1031F0004D3209F43196808308958827E00DF81F39
:10320000E00FF81F80830895040F151F261F371F36
:103210000895041B150B260B370B0895041715078B
:10322000260737070895000F111F221F331F089527
:1032300000951095209530950F5F1F4F2F4F3F4FF2
:103240000895019110810EC0019111912191308159
:103250000BC00191108117FF05C03FEF2FEF04C095
:10326000008111272227332737FF03C0E1DF8DE2DA
:103270008D93CF93DF93CF92DF92EF92AA24BB245A
:10328000CC24DD24EE2440E2CAE0DD2755E093E3C0
:103290008881890F87FD9F7083FD907F891B8993AB
:1032A0005A95A9F7C0DFAA1CBB1CCC1CDD1CEE1C68
:1032B0004A9551F7E894EFE0FF2782910ED0EB306A
:1032C000E0F71EF068948A2D0CD088278D93EF903C
:1032D000DF90CF90DF91CF910895982F829501D004
:1032E000892F8F70805D26F0803309F408956894EB
:1032F0008D93089588278D93089581918D938823C8
:10330000E1F7089594E081918D939A95E1F70895FE
:1033100009919191992351F08A95D9F7319781912B
:103320008D930A9519F08823D1F70895E3CFFF9381
:103330005527F8E0469508F4500F57954795FA95AC
:10334000D1F7FF910895FF93881BF9E0001FFA95CC
:1033500011F4FF910895881F841B18F4840F88943A
:10336000F5CF0894F3CF8FEF83959D919923E1F7E3
:103370000895F9DC0F770895F6DCFFDC0395AAF0D9
:1033800087E1DD0CEE1CFF1C8A9589F00A95CAF7CF
:10339000FF205AF000240D280E280F28002039F0B5
:1033A0000A95DD0CEE1CFF1CDAF70A95F8CC84CDEB
:1033B000DADC85E041D10F7723E839EF42E25EE3C2
:1033C0009DDDDBDF25DD139727D08A3F40F00068C5
:1033D0008D3F18F4CDDD80E803C057D1CFDD8827BD
:1033E00084831BDD8BDD14DD139729EA3EE64CE96F
:1033F00052EC84DD22E332E541E852E40AD122EDC9
:1034000032EE4DE951EC05D120E93FEF4FE75FE3A4
:10341000B5DD848108271DC1802F9F2D991F881F2E
:10342000991F881F089548CD9EDC0023E2F320DE1B
:1034300019F43BDD0068089585E0FED0FF0C001F05
:1034400004830FE70695F79420D1506897DDE0DC00
:10345000139721E438E743ED5BEB50DD27E831EDCE
:1034600043E15DE3D6D02EE03CE343EC5DEBD1D00D
:1034700022E83DEA4BE25EE3CCD02CEE32E846E7B0
:103480005EEBC7D020E931EE49EA5EE3C2D020E826
:103490003FEE4FEF5EEBBDD024EC3FEF4FE75FE335
:1034A000B8D0B6DC139784818F5799F02AF4D82EC0
:1034B0000FEFE02EF02E04C0D82EEE24FF240027BC
:1034C00076DC28E132E741E35FE318DD51DC349735
:1034D00055DDBFC048DC80E003C045DC802F80782C
:1034E000882321F0DF92EF92FF920F938F9345DCB8
:1034F000802F839512F4E0DC1BC080958A95885E4E
:103500000AF415C088501AF40CD0D92210C0DD245A
:1035100088501AF406D0E9220AC0EE2402D0F9221B
:1035200006C09FEF8770990F8A95EAF7089537DCF8
:103530008F918823D9F35F914F913F912F910F93F2
:1035400081DD0F9199F390F3A0D0506817CDADDCD9
:1035500080C009DC86E070D005830F772BE33AEA60
:1035600048EB5FE3CBDC54DC139741D028F4858132
:1035700088236AF7A1DC6DC08F778483F4DB3497EE
:10358000FCDE46DC139723E632E446E357EBB6DC79
:1035900029ED37EA4AE159E33CD026E538E14EEA25
:1035A0005AEB37D026E53CE84DE15CE332D02DEC18
:1035B00037E543E65DEB2DD02DEE3DEF45E75EE3CD
:1035C00028D028E132E741E35FEB23D05ED0D6DCA0
:1035D00024DCDD24EE24FF2404818FE7080F069508
:1035E000F79436DC8581881F08F424DC32C0C5DB03
:1035F0008827039512F48894089507301AF0812FD4
:1036000008940895FF1C881F0A95E2F7812B88947F
:103610000895B4DCADDB349771CCA5DB0F93AF9389
:10362000BF930F7702DFFF91EF91A2DB67DC92DFA0
:103630008F918078082B08950FB6F8944A925A9289
:10364000E42DF52DA42DB52D480E8827581E0FBE4C
:1036500008950FB6F894599049900FBE089583DBF2
:10366000002331F02BED3FE049EC5FEB87DCA1CE8E
:1036700023CC79DB802FFF0C001F901728F4091B47
:10368000881F0795F794089517CC5FE340E8332728
:103690002227089568DB0F930F776ADC1FDF8F9175
:1036A0008078082B089508CC5EDB0023E2F3D9F381
:1036B00088E0C2DFADDB1196FF0C001F8FE7080F1B
:1036C0000795F7940695F79483E08F93A6DBA0DB2C
:1036D000139749DBBDDB4CDB389750DC91E0CADF48
:1036E0008F918A9511F08F93F1CFB3CF8EE3380E7F
:1036F000C1166C01AD68240011A40300355D000003
:10370000906500000000E4420AD71F41000000005D
:10371000000020C100007A440000C842FB3A703D1E
:103720000000F0415839343E0000A0410000204123
:103730000000803F1B2F654200000040000048420F
:103740003F2F5E76202E2D40252630313233343502
:10375000363738394142434445464748494A4B4C3D
:103760004D4E4F505152535455565758595A0000C8
:103770002020202020202020202020202020202049
:103780002020000020484920000020002D2D2D2E53
:103790002D002E2E2E2E2E00260025004000480043
:1037A000330032003100495733484556202F20500E
:1037B0004133434B5200414E54454E4E4120414E01
:1037C000414C59534552000056302E33312053504E
:0637D0003353574A0000CC
:00000001FF
